S3150004000000000000000000000000000000000000E6
S3151C0000005CF09FE55CF09FE55CF09FE55CF09FE58E
S3151C0000105CF09FE500F020E358F09FE504F05EE2FB
S3151C00002000F020E304F05EE200F020E304F05EE260
S3151C00003000F020E3180050E30300001A38009FE587
S3151C000040000051E10000001A14F09FE500F05EE28A
S3151C00005000F020E304F05EE200F020E304F05EE230
S3151C00006000F020E31005001C2C00001C3400001CB2
S3151C0000705400001C5C00001C2400001C260002000E
S3151C0000800000A0E1010000FA1FB51FBD10B510BD90
S3151C000090DFF80CD0FFF7F8FF00F058E900F0FFF985
S3151C0000A01080040003B4FFF7F1FF03BC00F0FEF957
S3151C0000B0F0402DE90040A0E10150A0E10260A0E162
S3151C0000C014709DE5090054E304F18F30200000EA0A
S3151C0000D01F0000EA060000EA080000EA0A0000EA1F
S3151C0000E00C0000EA0E0000EA100000EA120000EA0A
S3151C0000F0140000EA00F020E3F0119FE5170000EA67
S3151C00010000F020E3E8119FE5140000EA00F020E36C
S3151C000110E0119FE5110000EA00F020E3D8119FE5ED
S3151C0001200E0000EA00F020E3D0119FE50B0000EA68
S3151C00013000F020E3C8119FE5080000EA00F020E368
S3151C000140C0119FE5050000EA00F020E3B8119FE509
S3151C000150020000EA00F020E30300E0E3F080BDE8C3
S3151C00016000F020E3080091E58000C0E3080081E56B
S3151C0001700100A0E30C0081E50020A0E3010056E38A
S3151C0001800000001A402082E3000053E30000000A2E
S3151C000190012082E3000057E30400000A040057E331
S3151C0001A00500000A080057E30900001A050000EACA
S3151C0001B000F020E30C20C2E3080000EA00F020E374
S3151C0001C0042082E3050000EA00F020E3082082E315
S3151C0001D0020000EA00F020E30300E0E3DEFFFFEA92
S3151C0001E000F020E3022082E3005081E5082081E52F
S3151C0001F0080091E5800080E3080081E50000A0E38B
S3151C000200D5FFFFEA38402DE90040A0E10800A0E335
S3151C0002100030A0E30320A0E10010E0E300008DE520
S3151C0002200400A0E1A1FFFFEB3880BDE810402DE9DA
S3151C0002300020A0E10130A0E1090052E302F18F3059
S3151C000240200000EA1F0000EA060000EA080000EA97
S3151C0002500A0000EA0C0000EA0E0000EA100000EAA0
S3151C000260120000EA140000EA00F020E37C109FE56F
S3151C000270170000EA00F020E374109FE5140000EA62
S3151C00028000F020E36C109FE5110000EA00F020E36B
S3151C00029064109FE50E0000EA00F020E35C109FE569
S3151C0002A00B0000EA00F020E354109FE5080000EA6A
S3151C0002B000F020E34C109FE5050000EA00F020E367
S3151C0002C044109FE5020000EA00F020E30300E0E38F
S3151C0002D01080BDE800F020E3040091E50040E0E357
S3151C0002E0000044E0000083E50000A0E3F7FFFFEAFE
S3151C0002F00020230320202303003023032030230364
S3151C0003000060230320602303007023032070230353
S3151C00031038402DE9AC009FE5004090E50F0A04E249
S3151C000320020950E30700000A00F020E30D10A0E1CB
S3151C0003300100A0E3BCFFFFEB301507E300009DE5C1
S3151C000340010050E1F8FFFF3A3880BDE878409FE590
S3151C00035078509FE578009FE54E1700EB921700EB4F
S3151C000360000094E5000050E30000000AA90000EB21
S3151C000370000095E5C51700EB6800A0E3D71700EB56
S3151C000380782805E34C109FE54C009FE5160000EB12
S3151C000390002800E344109FE544009FE5120000EB93
S3151C0003A05EF07FF55EF07FF56EF07FF57500A0E3DD
S3151C0003B0CA1700EBD5FFFFEB0000A0E324109FE556
S3151C0003C0000081E5930000EBC01F240304100218F3
S3151C0003D0142F0118007E32012008001C0000320177
S3151C0003E00078001C007632010080320110402DE995
S3151C0003F0202052E20500003A1850B1E8202052E2B3
S3151C0004001850A0E81850B1E81850A0E8F9FFFF2AC8
S3151C00041002CEB0E11850B1281850A0281800B148D7
S3151C0004201800A0481040BDE802CFB0E1043091246A
S3151C000430043080241EFF2F01822FB0E1B230D12060
S3151C0004400120D144B230C0200120C0441EFF2FE140
S3151C0004504FF0000200B5134694469646203922BF3B
S3151C000460A0E80C50A0E80C50B1F12001BFF4F7AF86
S3151C000470090728BFA0E80C5048BF0CC05DF804EB68
S3151C000480890028BF40F8042B08BF704748BF20F8D6
S3151C000490022B11F0804F18BF00F8012B7047044641
S3151C0004A0AFF300802046FFF7FDFD00000149182030
S3151C0004B0ABDFFEE72600020070470000101F11EE9E
S3151C0004C0011AC1E30410C1E3021BC1E34FF07FF51F
S3151C0004D0101F01EE0EF0A0E180402DE90F70A0E385
S3151C0004E0071001E0121F06EE1F70E0E3070000E094
S3151C0004F0110F06EE3F7701E3073003E0913F06EE4E
S3151C0005000100A0E3820080E1510F06EE8080BDE869
S3151C000510DCD09FE50107A0E30217A0E30020A0E3BF
S3151C000520042080E4010050E1FCFFFFBAC4009FE5F3
S3151C0005300010E0E3001080E5BC009FE50A10A0E374
S3151C000540081080E50C1080E50020E0E3002080E523
S3151C000550801081E3081080E50050E0E398609FE579
S3151C00056098709FE5048096E5088045E0008087E545
S3151C000570D2F021E388D09FE553F021E30000A0E3ED
S3151C0005800010A0E31F20A0E32D3300E3D1FFFFEBF7
S3151C00059070009FE50110A0E31020A0E3053301E3E2
S3151C0005A0CCFFFFEB3206A0E30210A0E31220A0E36F
S3151C0005B0053301E3C7FFFFEB4C009FE50310A0E3E7
S3151C0005C00E20A0E3043301E3C2FFFFEB3C009FE5D2
S3151C0005D00410A0E30B20A0E3053301E3BDFFFFEBF2
S3151C0005E0100F11EE010080E3100F01EE20C09FE5F5
S3151C0005F01CFF2FE1108004001400080000202303B8
S3151C00060000102E01108404000000011800003201A5
S3151C000610008032018000001C0000A0E30010A0E353
S3151C0006200020A0E30030A0E30040A0E30050A0E3BC
S3151C0006300060A0E30070A0E30080A0E30090A0E3AC
S3151C00064000A0A0E300B0A0E310C09FE500F08CE57D
S3151C00065000F020E300F020E300F020E300F09CE52E
S3151C000660E80FFFFFB0FBF1F202FB110110467047C9
S3151C0006700000000000000000000000000000000058
S3151C0006800000000000000000000000000000000048
S3151C0006900000000000000000000000000000000038
S3151C0006A00000000000000000000000000000000028
S3151C0006B00000000000000000000000000000000018
S3151C0006C00000000000000000000000000000000008
S3151C0006D000000000000000000000000000000000F8
S3151C0006E000000000000000000000000000000000E8
S3151C0006F000000000000000000000000000000000D8
S3151C00070000000000000000000000000000000000C7
S3151C00071000000000000000000000000000000000B7
S3151C00072000000000000000000000000000000000A7
S3151C0007300000000000000000000000000000000097
S3151C0007400000000000000000000000000000000087
S3151C0007500000000000000000000000000000000077
S3151C0007600000000000000000000000000000000067
S3151C0007700000000000000000000000000000000057
S3151C0007800000000000000000000000000000000047
S3151C0007900000000000000000000000000000000037
S3151C0007A00000000000000000000000000000000027
S3151C0007B00000000000000000000000000000000017
S3151C0007C00000000000000000000000000000000007
S3151C0007D000000000000000000000000000000000F7
S3151C0007E000000000000000000000000000000000E7
S3151C0007F000000000000000000000000000000000D7
S3151C00080000000000000000000000000000000000C6
S3151C00081000000000000000000000000000000000B6
S3151C00082078640000C1000000BD030000BF03000087
S3151C0008300000000000000000000000000000000096
S3151C000840000000000000000000000000C1030000C2
S3151C0008500000000000000000C3030000EB000000C5
S3151C000860C5030000C5030000C5030000C503000046
S3151C000870C5030000C5030000C5030000C503000036
S3151C000880C5030000C5030000C5030000C503000026
S3151C000890C5030000C5030000C5030000C503000016
S3151C0008A0C5030000C5030000C5030000C503000006
S3151C0008B0C5030000C5030000C5030000C5030000F6
S3151C0008C0C5030000C5030000C5030000C5030000E6
S3151C0008D0C5030000C5030000C5030000C5030000D6
S3151C0008E00348854601F0FAF8004800472B0D000026
S3151C0008F07864000078490020486188610A69774954
S3151C0009004A61886107200861704770B5724D0026E0
S3151C0009102868401C2860000E00281AD02E606869C2
S3151C00092006E0C1680A0E0902090A5118C160C069AD
S3151C0009300028F6D10DE0E068296888420CD8E069E9
S3151C000940686186612269002160699047204601F032
S3151C000950E5F86C69002CEED161480020C04670BDDC
S3151C0009605E490869C2035C4801D50122C260C2689F
S3151C000970594889690069002A02D0411A081870472B
S3151C000980401A704754480069704770B5FFF7E8FF76
S3151C000990514E0546F06800281CD00023F3603269CE
S3151C0009A0B069AD1A07E0C1688A4202D8891AC160CB
S3151C0009B000E0C360C0690028F5D10BE0E068A842DE
S3151C0009C00BD82269002160699047E069B061204616
S3151C0009D001F0A4F8B469002CF0D170BD70B50646C0
S3151C0009E0FFF7BEFF3C4D04460A21286901F028F892
S3151C0009F0B16848432418202001F0BAF800281BD0FF
S3151C000A00B168816031690161716941617168002356
S3151C000A10C460C3614160A9680160491CA960A969D9
S3151C000A2000290CD00022CE68B4420AD2C161002A29
S3151C000A3005D0D061002070BD0020C04370BDA861E8
S3151C000A40F8E70A46C9690029EDD1D061C361F1E70F
S3151C000A5070B5064680680A2100F0F2FF1E4D296813
S3151C000A604418202001F084F8002817D0B168816052
S3151C000A7031690161716941617168C460416069686D
S3151C000A800160491C696069690026002909D0CA6889
S3151C000A90002394421AD2C16168611AE00020C04347
S3151C000AA070BD8661C661F7E7CA69002A08D0D3689B
S3151C000AB09C4209D8C261CA699061C861816108E01B
S3151C000AC0C661C861836104E00B461146CA6894423C
S3151C000AD0EAD2002070BD0000CC13000000E000E04C
S3151C000AE02C14000008B50821002300911A46591E33
S3151C000AF000F026F808BD00B5030001F001F8091E38
S3151C000B0006080B0D101215171E00304810E02F4852
S3151C000B1020300DE02E480BE02D48203008E02D48F3
S3151C000B2006E02C48203003E02B4801E02A48203000
S3151C000B304068C0430860002000BD0320C04300BDC0
S3151C000B40F0B504461E460320C043230000F0D8FF20
S3151C000B50093706080B0D1012151737001B4C10E031
S3151C000B601A4C20340DE01A4C0BE0194C203408E0CA
S3151C000B70184C06E0174C203403E0174C01E0164CC9
S3151C000B802034A56880239D43A5600127E7600025C6
S3151C000B90012A00D14025002E00D03D43059A002A8B
S3151C000BA00ED0042A0FD0082A09D10820054302209A
S3151C000BB005432160A560A0681843A0600020F0BD15
S3151C000BC00C208543F3E70420F0E7000000202303F4
S3151C000BD0003023030060230300702303FEE7FEE7B7
S3151C000BE0FEE7FEE7FEE7000004490968016070475E
S3151C000BF010B52022024900F04DFF10BD74580000AC
S3151C000C00E01700008F4A131D106019600020704702
S3151C000C10F0B58C4F0D4684468B488C498C4E3C1D3A
S3151C000C20FFF7F0FF002818DB874838600821C94306
S3151C000C30864801E0761E11D022688242FAD16246AD
S3151C000C403A6022682A60824A03E023682B60521E9F
S3151C000C5004D02B688342F8D00020F0BD0846F0BDB6
S3151C000C6038B50D46002100910121C906014376487D
S3151C000C70784C2430FFF7C6FF002818DBA00629187D
S3151C000C80714D28352846FFF7BDFF00280FDB694646
S3151C000C902846FFF7BDFF002809DB0098641E0028C4
S3151C000CA002DA002CF3D103E0002C01D0002038BD61
S3151C000CB00820C04338BDFCB50D46002100910191AA
S3151C000CC00121C90601436048624C2430FFF79AFF94
S3151C000CD0002822DB5C4E610628363046FFF792FF61
S3151C000CE000281ADB371D69463046FFF791FF00289E
S3151C000CF013DB01A93846FFF78BFF00280DDB009894
S3151C000D00641E400002D40198002802DB002CEAD1A4
S3151C000D1004E0002C02D028800020FCBD4E48288010
S3151C000D200820C043FCBDFEB50C4681B2000C4B4FDF
S3151C000D30D21C029101909508454E69463846FFF72C
S3151C000D40BAFF002843DB6846018803200002814362
S3151C000D50FF2001300143684601803846FFF780FFBB
S3151C000D60002834DB3D486946401CFFF7A4FF0028D9
S3151C000D702DDB68460088C00725D0002E25D0694685
S3151C000D803846FFF798FF002821DB6846018834485F
S3151C000D90014034480143684601803846FFF760FF2E
S3151C000DA0002814DB2D480299801CFFF759FF0028E8
S3151C000DB00DDB2A480199C01CFFF752FF274E361D32
S3151C000DC0002804DB14E0761ECCD10820C043FEBDEF
S3151C000DD0208881B23046FFF743FF0028F7DB2068E6
S3151C000DE0010C3046FFF73CFF0028F0DB241D6D1E6E
S3151C000DF0002DEDD10020FEBDF0B58C4601461A48EB
S3151C000E00002515E04A5D030A5A4000242346174F65
S3151C000E1007E0D60702D05E00BE5B74405B1C9BB22B
S3151C000E205208002AF5D1000244406D1CA0B2ADB296
S3151C000E306545E7D3F0BD0146401E80B20029FAD1B4
S3151C000E4070470000202101180C1100004E3C2B1A83
S3151C000E5010270000A0860100ADDE000002D20000B3
S3151C000E60FCEFFFFF01100000FFFF0000BC13000099
S3151C000E7070B5644C0146503103C4FF3145312160C5
S3151C000E800821616001460022FF3181310A614A61F5
S3151C000E908A61026201685C4D5C4E083CA94202D123
S3151C000EA04168B14206D00121490200F00CFE2068BF
S3151C000EB00560466070BD53490246903205C1FF303D
S3151C000EC0993008601020486070474E480068C16819
S3151C000ED0491CC16070474B4800680169491C016187
S3151C000EE07047484800684169491C4161704745483C
S3151C000EF000688169491C8161704742480068FF305F
S3151C000F0081308169016270473E490968FF31813130
S3151C000F10086270473B480068FF308130016A816176
S3151C000F20704710B53748016801200831FFF7E3FD0B
S3151C000F3010BD70B5334D0646FF202C689D300059F8
S3151C000F40052100F07DFD8800001946622868FF30E7
S3151C000F508130C169491CC16170BD10B5294CA1689D
S3151C000F600B68E2680968521E934204D909040143BE
S3151C000F702068016210BDCA0061688850A0680068BC
S3151C000F80C00041180120091DFFF7B5FDA0680168C6
S3151C000F90491C016010BD30B51A4C22681346FF323D
S3151C000FA081321569082D04D311690904014319629C
S3151C000FB030BD1269D200D218FF3201321065FF22F1
S3151C000FC0206891321258D2001018FF30013041654A
S3151C000FD02068FF3081300169491C016130BD10B5A4
S3151C000FE0084C2268D369090480B21B070143980E7A
S3151C000FF08018FF30013001612068C169491CC1613C
S3151C00100010BD0000E813000043415254474F4C45A5
S3151C001010F8B5FA4D0126FA4C76021421284600F042
S3151C00102052FD2068F749884252D16168F6488142D0
S3151C0010304ED1A06800284BD1E068002848D1206911
S3151C0010400421F24A904204D1F1486169A26906C0A2
S3151C001050072188002058EF4FEF4BF04AB84210D1B9
S3151C001060491C880000196860A868401CA860C91C37
S3151C001070880027589F4204D02058904201D0B14284
S3151C001080F2DB8800205898420DD1491C88000019B3
S3151C001090E8602869401C2861C91C880020589042B9
S3151C0010A001D0B142F5DB761EB14208DC880023581C
S3151C0010B0934204D100194268D348824208D00020CA
S3151C0010C028606860E860B520FFF789FFB520F8BD89
S3151C0010D00020F8BDF8B50020CD4C00900834E0691E
S3151C0010E0006800908007FAD5F420FFF736FFCC4A3B
S3151C0010F0E0690068114600908143F9D1FB20FFF797
S3151C0011002CFFC84D69462846FFF782FD010002D018
S3151C001110FF2404346AE000993C24214328460091AC
S3151C001120FFF770FD010002D0FF2406345EE0BE4EC0
S3151C00113069463046FFF76CFD010002D0FF240934D6
S3151C00114054E0BA48009901401120014330460091F1
S3151C001150FFF758FD010002D0FF240C3446E011268F
S3151C001160B60169463046FFF753FD010002D0FF2445
S3151C0011700F343BE00098010909010B20014330465E
S3151C0011800091FFF73FFD010002D0FF2412342DE031
S3151C0011904721802689016120770180010091FFF794
S3151C0011A031FD010002D0FF241A341FE00099612092
S3151C0011B0B143B94380010091FFF724FD010002D021
S3151C0011C0FF241D3412E069462846FFF721FD010065
S3151C0011D002D0FF24253409E000992846A14300913A
S3151C0011E0FFF710FD010006D0FF2427342046FFF729
S3151C0011F0F6FE2046F8BD0020F8BDF8B5002000908C
S3151C001200834801680805040F082C02D8601E044296
S3151C00121003D02146FF24613445E07D4A083210691B
S3151C001220002C13D103685B0C9B0703D00268520386
S3151C001230940F0BE003687B4C1B041B0D203CA34244
S3151C00124003D192681268012A08D0042409060D0FDE
S3151C001250032D05D9FF242946713424E00224F5E721
S3151C001260002D08D10168C90C890703D00068C0028B
S3151C001270850F00E003256C4E69463046FFF7C8FC17
S3151C001280010002D0FF247B340DE000982101400AA6
S3151C00129040022943014330460091FFF7B3FC01008D
S3151C0012A006D0FF247E342046FFF799FE2046F8BD63
S3151C0012B00020F8BDF0B59C465D4B91B01C680746F6
S3151C0012C06408169E179864001C600B04BC330093BC
S3151C0012D0AF23090C9B04C918029203250191012214
S3151C0012E03346002101E05B08491C012BFBD10E2370
S3151C0012F09A434907090F1143F023421E99431307CA
S3151C0013001B0F1C010C430721090201228C435202AC
S3151C00131014438C4351018C430C433146002201E09B
S3151C0013204908521C0129FBD10721C9038C435107CB
S3151C0013308A0B22430F2189048A43990411430722ED
S3151C001340920591430122D20511430722520691436D
S3151C0013500A04FF32AB006C46BD32E250354A090C1A
S3151C00136089186D1CAA00A15031464143604640189D
S3151C001370401E6D1C00F064FB000211214904203044
S3151C0013800843A90060506D1CA9002B4860506D1CB9
S3151C001390A9002A4860506D1C3420A90060507807AB
S3151C0013A0400DA03001043802014325489922816072
S3151C0013B0694652048918C1600021416021490868A8
S3151C0013C00007000FFBD111B0F0BDFEB5064600208C
S3151C0013D06946088169201C4601214002FFF740FC32
S3151C0013E0010002D08D24A400A8E009211648FFF7AD
S3151C0013F037FC01002CD0154CA0E00000EC75000059
S3151C0014000076000045494350534752414C525443C1
S3151C001410F81300004C45525054534F50444E45004F
S3151C001420BE03000068080000DC04000000F3FFFF98
S3151C001430000811180000181804083C023806181871
S3151C001440000D02180001021801D20000350200002E
S3151C0014500121F948FFF704FC010001D0F74C6DE0AF
S3151C001460F74D286900680004000F082815D0286865
S3151C0014700168012211430160992040043118102390
S3151C001480082001930090EF4A23460020FFF712FF25
S3151C00149001000CD0E94C153450E0224631460020A0
S3151C0014A0FFF741FC010041D0E44CE41D46E0E64C4C
S3151C0014B0686821460268D20602D4491E0029F9DC56
S3151C0014C000290AD0DC4E01211D363046FFF7C8FB29
S3151C0014D0010005D01324640130E0D84C23342DE0E0
S3151C0014E0D54F1E3702A93846FFF7E5FB010002D08F
S3151C0014F09924A40022E068460089000602D4641ED2
S3151C001500002CEFDC002C08D000213046FFF7A8FB8E
S3151C001510010006D0C94C3B3410E02146C74C383478
S3151C0015200CE0286801684908490001600021C2488E
S3151C001530FFF796FB010006D00524E4012046FFF7C1
S3151C0015404EFD2046FEBD0020FEBD90B0002005903D
S3151C0015503F204002FFF7AFFCFFF7BDFCB748C43085
S3151C001560FFF7FBFC0320FFF7CFFCFFF751FD01271C
S3151C001570B34C0546002803D0B04E0146C93623E0BD
S3151C001580AF4EAE48083ECC303168FFF704FD2069EB
S3151C0015900068AE490004000D884208D100F0CFF85F
S3151C0015A0010004D0D120FFF71AFDD12507E03078C1
S3151C0015B0C00703D1A06A0168394301600025002DCC
S3151C0015C008D0C1262946B6003046FFF708FD280478
S3151C0015D0801924E09948D030FFF7BFFC05A8FFF717
S3151C0015E003FB07A8FFF704FB099881B20598FFF7D0
S3151C0015F003FC0A990546A94203D0904E0146D936EA
S3151C001600E2E730784008C0070CD1E0690068800723
S3151C001610C10F07D08948DF30FFF7E1FC8C48E16831
S3151C001620086065E08548E330FFF797FCFFF765FC2B
S3151C0016308248E830FFF791FCFFF74CFD050003D00C
S3151C0016407E4E0146EB36BFE77C48EC30FFF785FC47
S3151C00165000F03BF9050003D0784E0146EF36B3E7A0
S3151C0016607648F130FFF779FC00F0D1F8050003D07D
S3151C001670724E0146F436A7E7CB208000FFF76DFCBF
S3151C00168014220AA9684600F005FA07A90EC905988E
S3151C001690FFF79BFE050003D0684E0146F93693E71B
S3151C0016A06648FB30FFF759FC00F044F9050003D0EF
S3151C0016B0CD260146B60087E76648FFF74EFCFFF7C6
S3151C0016C09CFD010005D0FF25C9352846FFF787FC80
S3151C0016D002E000F071F80546002D03D05D4E294648
S3151C0016E0F61C71E7E06807605A480830FFF735FCBE
S3151C0016F0FFF7F7FBE0680068012801D0FFF7F7FB4E
S3151C0017000025554E10E03146284600F0AFF96D1CF9
S3151C001710002911D000BF00BF00BF00BF00BF00BF23
S3151C00172000BF00BF00BF00BFE06900684008C007DB
S3151C001730E9D1FFF7EFFB7BE7FFF7F3FBF4E770B5A7
S3151C00174005220021120719203F4B4005C2600322C7
S3151C00175012030261424A414DD56042481061102075
S3151C0017605061012414600820C04302E0491C9942C0
S3151C00177021DA1668B607F9D5D5603B491161FF21F8
S3151C00178051611460002102E0491C994213DA156864
S3151C001790AD07F9D53549D16035491161C721890095
S3151C0017A051611460002102E0491C994203DA146855
S3151C0017B0A407F9D5002070BD70B52E4E3569F468A6
S3151C0017C01FE0206801280AD0002814D03069FF24A5
S3151C0017D0411B98342046FFF702FC204670BD208929
S3151C0017E081B26068FFF73CFA002808D03069FF24F4
S3151C0017F0411B9234EEE7A1686068FFF703FA0C34CC
S3151C0018006D1E002C01D0002DDBDC002070BD10B538
S3151C0018101320A0210002FFF723FA010002D0FF24A7
S3151C001820AD344AE04521C9011348FFF719FA0100F6
S3151C00183024D0FF24B03440E00CD200003602000055
S3151C001840001400000000041910270000870B00007C
S3151C0018501503010036030000A0860100000238347F
S3151C001860000021030001000200030002000258349C
S3151C00187000140202EC750000B0D000000921684873
S3151C001880FFF7EEF9010002D0FF24B13415E06548DC
S3151C00189001690968644A0904090D914212D18068DC
S3151C0018A0006811280ED15E48012189026F30FFF7AE
S3151C0018B0D7F9010006D0FF24B8342046FFF78FFB6A
S3151C0018C0204610BD00F080F810BD70B5554C206840
S3151C0018D0016804252943016000215448FFF7C0F91B
S3151C0018E0010001D0524C16E05148401CFFF735FB55
S3151C0018F04E4800210B38FFF7B3F9010002D0A5248E
S3151C001900A40008E0692000214002FFF7A9F90100A4
S3151C00191006D0474CE41C2046FFF761FB204670BDF1
S3151C0019207D20C000FFF787FA20680168A943016083
S3151C001930002070BD38B50020694608806920032147
S3151C0019404002FFF78DF9010002D0394C1C3436E0F9
S3151C001950364838491930FFF783F9010002D0344C58
S3151C00196023342CE0314D002124352846FFF778F925
S3151C001970010002D05724E40021E02C480B210B382F
S3151C001980FFF76EF9010002D0294C2C3417E02A4CC3
S3151C00199069462846FFF78FF9010002D0244C3434DF
S3151C0019A00DE068460088002802D1641E002CEFDC7E
S3151C0019B0002C01D0002038BD21461D4C3B3420464E
S3151C0019C0FFF70DFB204638BD70B51C4EB568746814
S3151C0019D01FE0206801280AD0002814D0B068FF2414
S3151C0019E0411B3F342046FFF7FAFA204670BD20897A
S3151C0019F081B26068FFF734F9002808D0B068FF246C
S3151C001A00411B3A34EEE7A1686068FFF7FBF80C341B
S3151C001A106D1E002C01D0002DDBDC002070BD0000EB
S3151C001A20B1D0000000140000790800000CD20000A0
S3151C001A30920200000183000010270000EC750000D4
S3151C001A4030B50B46014600202022012409E00D4634
S3151C001A50D5409D4205D31D469540491B25469540BC
S3151C001A6040191546521E002DF1DC30BD70B5002400
S3151C001A702546002801DA01244042002901DA012505
S3151C001A804942FFF7DDFFAC4200D04042002C00D09B
S3151C001A90494270BD03460B439B0703D009E008C9A6
S3151C001AA0121F08C0042AFAD203E00B780370401CEC
S3151C001AB0491C521EF9D27047D2B201E00270401C7A
S3151C001AC0491EFBD270470022F6E710B513460A469C
S3151C001AD004461946FFF7F0FF204610BD064C0125AB
S3151C001AE0064E05E0E36807CC2B430C3C98471034A4
S3151C001AF0B442F7D3FEF7F8FECC130000CC1300005B
S3151C001B0030B47446641E2578641CAB4200D21D4654
S3151C001B10635D5B00E31830BC1847000010B5002855
S3151C001B2023D0124B0022001F196803E0814203D800
S3151C001B300A4649680029F9D1002A0AD01368841A72
S3151C001B409C4204D1006818181060104602E05060D0
S3151C001B5000E01860002907D002680B1A934203D1D3
S3151C001B600B68D21802604968416010BD3014000031
S3151C001B70F0B50B30C108C900144F0026144A0FE0FB
S3151C001B8003688B420BD38B4205D95C1A43184568F4
S3151C001B9030C3083B00E04368136002C004E0021D2A
S3151C001BA010680028ECD13046002803D1386800287C
S3151C001BB001D00020F0BD064A06481060064A121ADB
S3151C001BC0D208D20044C001203860D7E73414000084
S3151C001BD0301400007C58000078640000211042205C
S3151C001BE08440088131126224C44888910000000098
S3151C001BF0000000000000000000000000A0EB8200B6
S3151C001C0000000000000000000000000000000000B2
S3151C001C1000000000000000000000000000000000A2
S3151C001C200864101800651018041024030410021808
S3151C001C30C01F24034880000068800000142F011870
S3151C001C40302F0118382F0118542F011800000000DE
S3151C001C500000000000000000000000000000000062
S3151C001C600000000000000000000000000000000052
S3151C001C700000000000000000000000000000000042
S3151C001C800000000000000000000000000000000032
S3151C0020004945435007000200744000004A0700007F
S3151C002010443130325F30420000000000221119208A
S3151C002020F00B002043020000B9390000C73900003C
S3151C002030000000000000000000000000000000007E
S3151C002040000000000000000000000000D539000060
S3151C002050000000000000000029020000E339000017
S3151C002060F1390000FF3900003D3A00003D3A0000FE
S3151C0020700D3A0000133A0000193A00001F3A0000FE
S3151C002080253A00002B3A0000313A0000373A00008E
S3151C0020903D3A00003D3A00003D3A00003D3A000042
S3151C0020A03D3A00003D3A00003D3A00003D3A000032
S3151C0020B03D3A00003D3A00003D3A00003D3A000022
S3151C0020C03D3A00003D3A00003D3A00003D3A000012
S3151C0020D03D3A00003D3A00003D3A00003D3A000002
S3151C0020E000000000000000000000000000000000CE
S3151C0020F000000000000000000000000000000000BE
S3151C00210000000000000000000000000000000000AD
S3151C002110000000000000000000000000000000009D
S3151C002120496E66360B02D10000030001042600012D
S3151C0021300001002000040020000000000005002013
S3151C002140080000008000000028040020000A00206F
S3151C00215000000000000000000000000048040020F1
S3151C002160000000000000000000000000000000004D
S3151C002170000000000000000000000000000000003D
S3151C002180010000000000000000000000000000002C
S3151C002190000000000000000000000000000000001D
S3151C0021A000F002F800F03EF80CA030C808382418DD
S3151C0021B02D18A246671EAB4654465D46AC4201D15D
S3151C0021C000F030F87E460F3E0FCCB6460126334251
S3151C0021D000D0FB1AA246AB4633431847843E000088
S3151C0021E0A43E0000103A02D378C878C1FAD8520728
S3151C0021F001D330C830C101D504680C60704700009B
S3151C0022000023002400250026103A01D378C1FBD8F0
S3151C002210520700D330C100D50B6070471FB51FBDD8
S3151C00222010B510BD03F09CFE1146FFF7F7FF00F03A
S3151C00223021F803F0B4FE03B4FFF7F2FF03BC00F071
S3151C00224017F8FEE7FEE7FEE7FEE7FEE7FEE7FEE71A
S3151C002250FEE7FEE7FEE7FEE7FEE7FEE7FEE7FEE734
S3151C002260FEE710B5FFF79CFF10BD0A4603467047F4
S3151C002270FEE77047FFF7FDFF03F040FC614E0027A9
S3151C0022803760052109077818306003F077FB03F0E7
S3151C0022900CFB03242407A08AB81EA08231685A4866
S3151C0022A008180782A08A2020C043A08231682020FB
S3151C0022B01322520289180880316853484030081886
S3151C0022C0408C524DC007C00F01D0022004E030687C
S3151C0022D04F494018808E000B287002F0C1FB03F09A
S3151C0022E03FFDA08AA7824B4A336890883546010B6E
S3151C0022F009030007000D0143907B0143424A9A18CB
S3151C0023001184464F4449396003223368520493436F
S3151C002310336000265EE038689221095CC022514376
S3151C0023204030818002F0F7FBA08A0120C043A082C6
S3151C0023302A680121344840301018018002F027FD1C
S3151C00234002F077FDA08A0720C043A08229680420DA
S3151C002350334A89188881A08A3248A08201202968BC
S3151C00236080032B4AC03A89180884A08A2E48A0826A
S3151C00237001212A6849032648803812185181A18AEE
S3151C0023802A49A18201212A68090312185181A18AAE
S3151C0023902749A18201212A68C90212185181A18AE2
S3151C0023A02449A18201212A688902101841813868B2
S3151C0023B003228030C07C520401021748081838607A
S3151C0023C08030807C296880079143400B0143761C32
S3151C0023D0F6B229600D48007886429CD303260E4C23
S3151C0023E0760400F029F838688030C07C0002001999
S3151C0023F038608030807C29688007B143400B0143DC
S3151C0024002960EEE78400002040A401008000002023
S3151C002410C0A101000004002000050020900000203F
S3151C00242040A30100FFBF0000FFDF0000FFEF00001C
S3151C002430FFF70000FFFB0000FEB5FE4D00262868D6
S3151C0024408030807C002817D10F273F0303F038FA11
S3151C002450F94C000C2168090C401AB8420CDDF748EF
S3151C002460FF218170F02141700670032003F0D2FB1E
S3151C00247020683904401820602968F14C8031887A1C
S3151C002480C87222680D2040031018808FC20A8A72F7
S3151C0024900106C90F03D18006800E01F0C5FF28680E
S3151C0024A00090407C002809D0012831D002282DD06C
S3151C0024B003282ED004282FD0052830D000980021C0
S3151C0024C0403081740098226880308446007A400629
S3151C0024D0C017DC495118898F401C4907C917491C6C
S3151C0024E0D94D084276D00022A88A8420C043A882EF
S3151C0024F0D0072168000ED54BC918001D8885002001
S3151C002500002110280ED21F231B1A0DE000F06EFBB3
S3151C002510FEBD00F0E0FBFEBD01F006FDFEBD00F0B9
S3151C002520D0FEFEBD0346103BAE8ADBB2002A07D0A6
S3151C0025301F26F643AE822768C44EBE19F38506E0F5
S3151C002540C34EAE8227681E02C04BFB189E85BD4E2D
S3151C00255000232768BF193F8CFF05FF0F01D0491CBC
S3151C002560C9B25B1CDBB20A2BF3D3002804D00529A5
S3151C0025701DD81F2802D016E0052914D9A88A002ABE
S3151C00258008D01F20C043A88223681020AF495918C1
S3151C002590C8850CE0AE48A882012023680003AB491D
S3151C0025A05918888503E0401CC0B22028A8D3521CA9
S3151C0025B0D2B2022A98D3A88A0420C043A8822268D1
S3151C0025C00020A249511888856046007A402108439C
S3151C0025D06146087221689B480818008C9D4E800431
S3151C0025E0800F02286CD00098A030007800284BD0B1
S3151C0025F0236803215803800F00908E484904964A8D
S3151C0026008B430260002723602DE0A88A0120C0436B
S3151C002610A882226800200D2149035118488403F022
S3151C00262080F98E4803F059F98249002009688031E7
S3151C002630C87702F0DBFC7F4800220068A0210A5400
S3151C0026408030C07C03220102834852040818794951
S3151C00265008608030807C216880079143400B0143D1
S3151C0026607F1CFFB221607E4800788742CDD300983C
S3151C0026707949020252186F490A60032252042168E2
S3151C0026804004914301432160216870480818C08AA0
S3151C00269001076848090F00684030C1740121817424
S3151C0026A03079002800D03CE7A88A0F20C043A882B6
S3151C0026B023680F2265484030181842843171FEBDCC
S3151C0026C0307901280BD1A88A0F20C043A882226822
S3151C0026D007215E4840301018418400203071604646
S3151C0026E0C07A544E00286046807A02D0002805D055
S3151C0026F008E0002806D002212F2001E0022130200C
S3151C00270003F016FB316808468030827A002A3CD0DA
S3151C002710012A42D00227062A52D0082ACFD1427C4F
S3151C002720530716D404231A431A404274827C403140
S3151C002730897A12015118C07F09061030090CC0B2E3
S3151C002740014301910023022200973321012003F04B
S3151C00275079FA306801468031CA7F002A56D0012A90
S3151C00276066D0032A65D0042AA9D101214030817480
S3151C002770216834480918C989C90775D02168091800
S3151C002780C9898907C90F70D01FE100224274012034
S3151C0027904031887402F097FBFEBD002640318E74D2
S3151C0027A00221312003F0C4FA02F010F902F003FDF5
S3151C0027B0A88A2C48A8822168224808184680FEBD93
S3151C0027C0427C930715D43A433A404274827C40318A
S3151C0027D0897A12015118C07F09061030090CC0B243
S3151C0027E0014301910023022200973221012003F0AC
S3151C0027F029FA30688030C07F002804D00228DED138
S3151C00280002F09AFFFEBD02F037FEFEBDAA8A022226
S3151C002810D243AA8223680D2252039B185F84AB8A7B
S3151C0028200123DB43AB8224680023A21853841DE0DA
S3151C00283027E0A5E090000020880000208C000020E6
S3151C0028408400002080A401000000003000A10100CB
S3151C002850FFE000002004002000050020A0860100E7
S3151C00286080000020FF7F00009FE0A1E00122CA77C4
S3151C002870897C4030807A090108180006000C212149
S3151C002880B1E023685A4A9B18DB89DB071ED0CF7739
S3151C002890A88A2020C043A882226820200D21490333
S3151C0028A05118088403F058F8002801D103F039F8B0
S3151C0028B03068014602468032907C4031897A00019C
S3151C0028C040180006010CD07F303049E02368484A86
S3151C0028D09A18D2899207D20F20D0012240308274D6
S3151C0028E00420C877A88A4348A882910322684048D6
S3151C0028F01018418003F030F8002801D103F011F8BC
S3151C0029003068014602468032907C4031897A00014B
S3151C00291040180006010CD07F403021E003F01CF863
S3151C002920226833495118898F8907C917491C0842DF
S3151C00293021D0316808468030C777AA8A2022D24324
S3151C002940AA82246820220D235B03E3181A84827C46
S3151C0029504031897A120151180906C07F090C503082
S3151C002960C0B20143009701910023022233210120AA
S3151C00297003F068F9FEBD3168012040318874FEBD44
S3151C002980012240308274AA8A1B4AAA822468531CDC
S3151C002990174AA21853800422CA77897C807A0901B7
S3151C0029A008180006000C64211DE0A98A124901E0E2
S3151C0029B0A98A1049A982226800211018418002F0B8
S3151C0029C0A1FF316801208031C87730680146024674
S3151C0029D08032907C4031897A000140180006D17FF4
S3151C0029E0000C7031C9B2084300970190BCE7000087
S3151C0029F080A40100FFBF0000FF7F0000002816D046
S3151C002A00012815D0002140004008491C400049B24D
S3151C002A100028FADAC00DE0221040CA17D20E52184E
S3151C002A2052095201891A1F22511A4018C0B2704706
S3151C002A30E0207047F0B503242407A18AFE49A18231
S3151C002A40002801DD012100E00021FC4A8902FC4E20
S3151C002A50891832680D277F03D219118101230021A1
S3151C002A605B02454207E0A28AF64AA2823268D21964
S3151C002A701381491C49B2002801DB024600E02A46A4
S3151C002A808A42F0DCF0BDF0B5EF4853210068012303
S3151C002A90095C0D270324EB4A5B027F032407E84DE0
S3151C002AA000290CD02621415EE84E084611300CD078
S3151C002AB00F2917D0A08AA2822868C0190381A08A70
S3151C002AC0A2822868C01903811BE03E20C043FFF781
S3151C002AD0B1FF0120FFF7AEFFA08AFF20A0820120D4
S3151C002AE080020BE03E20C043FFF7A4FF0120FFF746
S3151C002AF0A1FFA08AFF20A0820120C0022968891993
S3151C002B008884D1480068C18C491CC184F0BD30B58D
S3151C002B1003200007818ACE4B8382C94900240D6895
S3151C002B20CA4AAD182C84848A83820C685B1CA21842
S3151C002B301384828A8022D2438282096880200D22D5
S3151C002B4052038918088430BDBD480068BF49401827
S3151C002B50808E800480164042704710B503210907F9
S3151C002B608A8A8A138A82404280060D22C00D52022E
S3151C002B708318B34A1468B5482418E3828B8AB44B6D
S3151C002B808B821268591C1018C18210BDAE48006891
S3151C002B908030807A062801D00020704701207047BB
S3151C002BA070B5A94800210468227FA37D9A4201D3EF
S3151C002BB0D01A02E0BF20C01A8018C5B2E08C632868
S3151C002BC001D10121C903BF2A01D3002000E0501CFA
S3151C002BD0C0B2834202D10126B60331439A4202D1C6
S3151C002BE00122520311432943A18270BD70B5FFF720
S3151C002BF0D7FF0546FFF7CAFF002863D0924C216811
S3151C002C00087DBB285ED226228A5E632A5AD04031B2
S3151C002C10CE7C8B488D498F4B002E16D010321F2A26
S3151C002C2002681DD856182822B25E00689202401807
S3151C002C30408DC0B21043FFF7E1FE024620684421D6
S3151C002C40095A007F08181A541CE0026856183022CC
S3151C002C50B25E006892024018408E8005800D07E027
S3151C002C6056182C22B25E006892024018C08DC0B263
S3151C002C701043FFF7C3FE014620684422125A007F08
S3151C002C801018195420680577FFF75EFF1F21C842EC
S3151C002C901CDC20684422125A047F00211219995404
S3151C002CA0017FBF2901D3002100E0491C01772621A1
S3151C002CB0415E1F2907DAFFF7E6FE1F20FFF74DFFCF
S3151C002CC0FFF725FF70BD6321C18470BDFFF73CFF74
S3151C002CD0401E40B2F2E7F0B5FFF762FF0746FFF76A
S3151C002CE055FF00286FD0584E3068017DBB296AD22B
S3151C002CF02621415E632966D04030C07C504C534D22
S3151C002D00544B00280BD0103120681F2912D84119AA
S3151C002D102820085E216880024919498D11E0206827
S3151C002D2041193020085E216880024919498E89059F
S3151C002D30890D07E041192C20085E2168800249197B
S3151C002D40C98DC9B20843FFF759FE014630684422B3
S3151C002D50125A007F10181954306826210777415ED5
S3151C002D601F2902DAFFF78FFE2BE04422125A00219C
S3151C002D70D2199954017FBF2901D3002100E0491CB7
S3151C002D800177FFF7E1FE1E27FF43B84224DD3068BA
S3151C002D904030C07C002817D00420FFF74BFE0320D0
S3151C002DA00007818AFF21818201202168400249197E
S3151C002DB088843068C784FFF7C7FE401E40B2FFF701
S3151C002DC0CCFEFFF7A4FEF0BD3E20C043FFF732FE4B
S3151C002DD00120FFF72FFEECE731686320C884F0BDA5
S3151C002DE010B502F06DFD1849020C09680887CA86E1
S3151C002DF088844A8410BD10B5114A1168164BC9182F
S3151C002E00898E00244904047048081168C918C98EA3
S3151C002E10084310BD10B503200007818AFF21043129
S3151C002E208182074A00211468084BE4182184848A8D
S3151C002E3081821468E41811E0808B000001200000D8
S3151C002E4084000020FFFD00009000002040A001002F
S3151C002E50FF7F00000001002080A101006184848A9C
S3151C002E6081821468E418A184848A81821068C0183F
S3151C002E70C18410BD70B50446FFF7CCFF03210907BA
S3151C002E80888AFE488882FE4AE3061568DB0E0D26F4
S3151C002E907603AD196B858B8AFA4B8B8216680D14DB
S3151C002EA0F94BF61835848D8AFF258D820125166807
S3151C002EB0AD02F618B5848D8A0325ED438D821668FE
S3151C002EC00325F318DD848B8A88821068EF49401825
S3151C002ED0C48570BDF0B51F20FFF7CCFF032000078B
S3151C002EE0818A3021C9438182E54910230C680D2251
S3151C002EF05203A4186384838AE54B838201230C68DE
S3151C002F009B02E44D64196384838A2023DB438382FA
S3151C002F100C682023A2181384828ADF4D85825E02E8
S3151C002F200B68DA4A403A9B189E81838ADB4F87825C
S3151C002F300C687300A418A381848A85820C68A41863
S3151C002F40A684848A87820C68A2189384828A0822A3
S3151C002F50D243828209680820CB4A403289180880ED
S3151C002F60F0BDF8B5CE4F26213868415E0C124DB225
S3151C002F7029461F313F2904D21F2C02DC1F21CC42BB
S3151C002F8009DA0122E1B2D2038918818280304470A9
S3151C002F9085700120F8BDFFF7D7FD01463868B84E8D
S3151C002FA04030417632680D2149035218928AC27309
S3151C002FB032685118898A091201742846FFF7CDFD1B
S3151C002FC0FFF788FF38685321095C00290DD00321BF
S3151C002FD010230907FF22DC4209DA63004033C3844D
S3151C002FE08B8A8A82012252020AE0C4840FE00F2CCB
S3151C002FF00BDD63003C3BC3848B8A8A820122D2028E
S3151C0030003368A14959188A8401E06100C184C08CC7
S3151C00301040B2FFF70FFD6846FFF7EDFEFFF7E0FE37
S3151C003020FFF775FD386801218182803044708570F8
S3151C0030300020F8BDF0B5924D29680D267603891936
S3151C003040898A032409120818400040B2411024073B
S3151C003050A08A8C480C30A08201202A684003921951
S3151C00306010810A068A48A28AA08205D52A680020F1
S3151C00307092191081494204E001202A6880029219A3
S3151C0030801081A08A7F20C043A0822A680120921941
S3151C003090108100200122834F520206E0A38AA782D8
S3151C0030A02B689B191A81401C40B28842F6DBF0BD86
S3151C0030B0F0B5734D29680D2676038919898A032470
S3151C0030C00818400040B240102407A18A6D490C31F3
S3151C0030D0A18201212A688903921911810306002104
S3151C0030E0002B6B4AA38AA28204DA2A6892191181E0
S3151C0030F0404204E001222B6892029B191A81684AFD
S3151C003100684F12684032937B01225202002B13D067
S3151C003110A18A7F21C943A1822B6801219B19198190
S3151C003120002106E0A38AA7822B689B191A81491CD9
S3151C00313049B28142F6DBF0BDA38A5B4BA3824006F3
S3151C0031400123400EDB02C0182B689B191881A08A2C
S3151C003150A782286880190281A08A53487F30A082E2
S3151C003160286880190181F0BD0F304010704710B5DA
S3151C003170032109078A8A8A138A82C0051122C00D77
S3151C003180520283183E4A14683F482418E3828B8AED
S3151C003190424B8B821268591C1018C18210BD10B587
S3151C0031A0032109078A8A8A138A82C0050922C00D4F
S3151C0031B092028318324A146833482418E3828B8A95
S3151C0031C0364B8B821268591C1018C18210BD10B563
S3151C0031D0334C2068C27D014653074031002B14DA5C
S3151C0031E092070DD4812141560F314810FFF7D7FFA6
S3151C0031F02168822008560F304010FFF7B8FF0DE0FB
S3151C0032000F200856FFF754FF08E019200856FFF751
S3151C003210A4FC216850200856FFF70CFF2068C07DCF
S3151C00322000070CD503200007818A0821C943818227
S3151C003230134908200968144A40328918088010BDB1
S3151C00324070B5064602F03CFB154D04462868223034
S3151C00325002F0C7FD01461020C141601A30602D687E
S3151C0032602846363002F0BDFD01461020C1410F48EC
S3151C0032706A7C611A407C052A1FD019E0E0FF000019
S3151C00328084000020F38F000040A0010000A501006F
S3151C003290FFFB000080A10100FFBF0000FF7F0000B4
S3151C0032A090000020FFFD000080F7000000040020B5
S3151C0032B04004884203D2012070BDC001F9E70020FA
S3151C0032C070BDF8B5F8480068808A000418D4032637
S3151C0032D03607B08AF54FB782F54C202122680D209F
S3151C0032E04003101841846846FFF7AAFF00250128F1
S3151C0032F007D0B08AB78221680D2040030818458480
S3151C003300F8BDFFF764FFE8480121006841745321AA
S3151C003310095C00290ED081221156E64A10311F295C
S3151C00332021680AD889182823CB5E990223689A1823
S3151C003330528D09E0058345830BE08B182C21595EC1
S3151C003340236889029A18D28DD2B211430A0C0283C1
S3151C0033504183D9498182F8BDF8B5D34FD74D396819
S3151C003360D34EA0314878D64CC00707D1A88AD54879
S3151C003370A88201203268C002121910810020C87070
S3151C003380FFF7EBFB3868A03040784006400F062854
S3151C00339001D101F02BFE3168C9480818848BFFF750
S3151C0033A039FD282C43D0502C43D0782C43D0A02C4C
S3151C0033B043D0C82C43D0F02C43D00020A98A8321AB
S3151C0033C0A98232680102BB481218D184A98ABE4957
S3151C0033D0A982BE49326812181184A98AFF21A982C2
S3151C0033E001213268890212189184A98A8021C94355
S3151C0033F0A98233688022B2495B181A84AB8AD343EC
S3151C003400AB8233681818C284A88A1F20C043A882BE
S3151C00341032680C20511848853868A121095C06229F
S3151C0034200907490F511A8C4080308484F8BD01204D
S3151C003430C4E70320C2E70520C0E70720BEE7092032
S3151C003440BCE70B20BAE700B5974900230968DB43A4
S3151C0034500A46A032D0700B8402239370002240319E
S3151C003460CA75FFF77AFBFFF752FB00BD8E48002199
S3151C0034700068017781758182A121095C8030CA09A7
S3151C003480818C002A00D04900C1840020DBE700B5EE
S3151C003490854900230968DB430A46A032D0700B8499
S3151C0034A00223937000224031CA75FFF756FBFFF7C3
S3151C0034B02EFB00BD10B51446411A09D040001A1B3C
S3151C0034C0504302F0A9FC401C4010201800B210BD4D
S3151C0034D0D018C10F08184010F8E7F1B5724FA1219A
S3151C0034E038680126095C00258C4609074A0F3146B7
S3151C0034F091404CB2017F827D82B0914201D38B1ADE
S3151C00350002E0BF239B1A5B189BB28382BF2901D39F
S3151C003510002700E04F1CFFB20097BA4203D10127D7
S3151C003520BF033B438382914204D1818A0122520309
S3151C003530114381821F21029AC943614F012A23D15B
S3151C0035408030C08C00281FD16046C0091CD0604644
S3151C003550C00700D020210846FFF76CFA5748818A1D
S3151C0035605B4981825048012200689202A030417852
S3151C003570C907C91789028A184D490968C9190A81D8
S3151C00358041784906490E4170494801684C4808185B
S3151C003590808F454BC20A1868014680318A72C98CD5
S3151C0035A0002975D0062A73D1017DBB2970D24049EA
S3151C0035B00A68404951183027CF5F0246A0329178DD
S3151C0035C004290FD80323D3560620002F03DB411AE8
S3151C0035D03046884003E0411A30468840404218185D
S3151C0035E0D07043E00023DB4305290BD0002F11DDEF
S3151C0035F02021415E00291FDB032151561F2917DAA2
S3151C003600491C13E003201056002F00DB0123C018B1
S3151C003610D07028E0002F0FDA2021415E002915DC2E
S3151C003620032151561F23D94202DD491ED1701AE0CF
S3151C0036304030C6754D0116E0032151564B011A4602
S3151C00364020322025455F3946284605E003201056C2
S3151C00365042011346203B3846FFF72CFF054612480D
S3151C00366000684030C6751048006807840E4800681C
S3151C0036700146A0318A780746521C8A704037FA7D6B
S3151C003680012A06D003200856FFF767FAFFF73FFA10
S3151C003690FEBDBA88037FD3180E4AD554009A02770A
S3151C0036A0BF2A19D3002318E090000020DFFF00007A
S3151C0036B08400002040A0010001EC00000000003046
S3151C0036C000A00100FFF70000F30F00000CB0000083
S3151C0036D0FFFB000000010020531CBF882D04BF18EF
S3151C0036E0F84A2D0ED55503778030C28C521E93B2E4
S3151C0036F0C3840022CA70029DF34A012D1AD04D784C
S3151C003700ED090ED0808C83420BD103200007838ADF
S3151C0037107C23DB438382ED4804230568EC48281888
S3151C003720C38403252D07A88AEA48A882002C1DDD20
S3151C00373001201CE003230D2500201B076D03012619
S3151C003740760207E09C8A9A82E04C246864192681DA
S3151C003750401CC0B24C786407A70F0124BC408442AD
S3151C003760F0DC03200856FFF792FEFEBD0020DA4B64
S3151C00377080021843D54B1E680D277F03F61930812E
S3151C003780012200205202664208E0AB8ACE4BAB8275
S3151C003790CE4B1B68DB191A81401CC0B2002C01DB06
S3151C0037A0234600E033468342EFDC03200856FFF72E
S3151C0037B04AFEFEBDF0B5C94E00243068847584826D
S3151C0037C0FFF728FB03252D07A88A0320A882BF4FD5
S3151C0037D03868BF494018C4843068A030C47020467D
S3151C0037E0FFF7BBF9A88ABB48A88239680D2040039D
S3151C0037F009180C81A98ABA49A98239680818048152
S3151C003800F0BD00B5B54900200968A031C870FFF7A6
S3151C003810A4F900BD10B5B14C002120680177817553
S3151C00382081820221A03081704078C00701D02020FF
S3151C00383001E01F20C043FFF7FDF803200007818A23
S3151C003840A8498182206801230246A03041789B0248
S3151C003850C907C9178902C9189C4B1B680D24640328
S3151C0038601B19198141788023194341704807810F20
S3151C0038704020C8408032D0840020FFF708FE10BDCF
S3151C003880F0B5FFF761F9954F3968403148761F202E
S3151C003890FFF763F98D4C20680D256D034019828A4C
S3151C0038A0396808464030C27322685219928A12122D
S3151C0038B002741E22D243CA84C07C002847D0022030
S3151C0038C0FFF7B8F8386800260685067786751F2028
S3151C0038D0FFF7D0FA39685320425C0007002A08D04B
S3151C0038E0828AFF228282012223685202784FDB19C8
S3151C0038F09A848E82818A2021C94381822268202152
S3151C00390052191184818A784D858201272268BF034A
S3151C003910764952189781828A754E86822368721C54
S3151C0039205B189A81838A858223685B189F84838AA5
S3151C0039308682236859188A84818A0821C943818210
S3151C00394021680820624A403289180880F0BD1F2071
S3151C003950C043FFF76FF80120B2E770B50446FFF7C6
S3151C00396059FA03210907888A624B8B82574AE0065B
S3151C0039701568C00E0D267603AD196885888A5E48C3
S3151C00398088825E4D16685248361835848D8AFF2506
S3151C0039908D8201251668AD0230188584888A8B8233
S3151C0039A01068524940314018C48570BD00B5FFF7F8
S3151C0039B0CBF84A4959220968505400200877887563
S3151C0039C01C20FFF7CAFF00BD70B5FFF700FCFFF710
S3151C0039D021FA03200007818A3021C94381823B4A90
S3151C0039E0002113680D2464031B195984838A3D4BDB
S3151C0039F083821368424D5B195984384B1B68D975F1
S3151C003A0099759982838A2023DB43838213681B1949
S3151C003A101984838A344D85821468344BE418A18139
S3151C003A20848A334E86821468E418A181848A85822E
S3151C003A301468E418A184848A86821068C01881845C
S3151C003A4070BD10B5002300281CD02E4C0022A042AD
S3151C003A5000D92046521C400052B20028FADAD4176C
S3151C003A60E40EA41864096401121B1F24A21AD2B204
S3151C003A700A70082A09D2000E0006A21AD040C0B24B
S3151C003A800B7010BD0B70002010BD000ED21F0A70EB
S3151C003A9010BDF0B503242407A18A0E49A182002873
S3151C003AA001DD012100E00021174A8902074E891811
S3151C003AB032680D277F03D2191181012300215B0275
S3151C003AC045422BE000010020FFFD00008400002081
S3151C003AD040A00100808B00000170000090000020B7
S3151C003AE0FFF70000FFFB0000FFBF0000C0A40100A1
S3151C003AF0FF7F0000E0FF0000F30F00000CB0000089
S3151C003B0080A10100FFFF7F0001400000A28AFE4A3F
S3151C003B10A2823268D2191381491C49B2002801DBE2
S3151C003B20024600E02A468A42F0DCF0BDF0B50E27BC
S3151C003B300022F64DF64EFF43F64C0F23002916D0F5
S3151C003B40002809D0104609E0296889198988890640
S3151C003B508916791AC184F0BD1F461846FFF71FFB4C
S3151C003B602068C17D0909C9438907EDD1F0BD00282C
S3151C003B7001D0104601E01F461846FFF7F8FA2868E0
S3151C003B8080194088216880068016381AC884F0BDC2
S3151C003B9040000F3840B2704730B5DE4C002021681B
S3151C003BA0DA4A08851068DA4BC018808880068016A9
S3151C003BB0FFF7EEFF2168803148701068C0184088F6
S3151C003BC080068016FFF7E4FF216801220B4680332E
S3151C003BD098709A56002A01DB154600E055420028CB
S3151C003BE001DB034600E043429D4203DD0B8D0425A9
S3151C003BF02B430B85002A03DD0A8D02231A430A85F3
S3151C003C00002803DD088D012210430885CA7D900615
S3151C003C10800F13D0012820D0022821D003280CD1D4
S3151C003C20088D01218007C00FFFF780FF2068008DDB
S3151C003C30C007C00F0021FFF779FF30BD2820085EA2
S3151C003C40042801DB012100E00021042802DB800797
S3151C003C50C00FF0E7C007C00FEDE7D007C00FE9E7BC
S3151C003C60D007C00F0121E6E7F8B5FEF76DFFA94C9A
S3151C003C70A64D21680A464032507628680D235B0300
S3151C003C80C018808AD0732868C018808A0027001242
S3151C003C9010748F82C87DA24E03079F489F4AB38A21
S3151C003CA0B08203D528688018078003E02B6808209B
S3151C003CB09A181080C87D4007400F030002F07AF95D
S3151C003CC008050E1B2F43435E66451F20FEF745FF66
S3151C003CD0216850200856FFF7ADF918E01E20C04396
S3151C003CE0FEF73BFF216850200856FFF7A3F921E099
S3151C003CF02168C88429E00020FEF72FFF2068403089
S3151C003D00C07C002805D00120C043FEF793FE1F206F
S3151C003D10EEE72020FEF78EFE0020C043F5E70020CC
S3151C003D20FEF71BFF20684030C07C002805D002200F
S3151C003D30FEF780FE1E20C043DAE71F20C043FEF7B5
S3151C003D4079FE0120F4E7FFF727FF2068C07D4007B6
S3151C003D502BD4FFF7BFF820685321095C002922D019
S3151C003D60C07D81071FD56D49C207FF204039002A37
S3151C003D70B28AB08212D00120400211E02020FFF747
S3151C003D8088FE0020C043FFF784FEC0E71F20C04307
S3151C003D90FFF77FFE0120FFF77CFECBE70120C00268
S3151C003DA02A6851188884FEF7B2FEFFF719F82068B6
S3151C003DB05E30FFF720F82068877507774787878767
S3151C003DC0F8BD10B501F07CFD524909688884000CC9
S3151C003DD0488410BD7CB5064608686946C008FFF7CE
S3151C003DE030FE4C4D442229684E4C525A0B7FD21839
S3151C003DF0A054087FBF2801D3BF2000E0401C0877D1
S3151C003E0001A93068FFF71DFE694609780A01694653
S3151C003E1009790A4329680B4640339D880E7FAD19E4
S3151C003E2062550A7FBF2A01D3BF2200E0521CD2B2C0
S3151C003E300A779B889A18A054087FBF2801D3BF20F5
S3151C003E4000E0401C08777CBD70B5324A0E2314680E
S3151C003E500025E3842D4B2E4C00292BD000281868F6
S3151C003E6011D00019808880068016FFF791FE116814
S3151C003E7081268E57B0421ADA186800198088800687
S3151C003E808016401C10E00019808880068016FFF7FB
S3151C003E907FFE116881268E57B04208DD186800190E
S3151C003EA0808880068016401EFFF779F970BD106861
S3151C003EB0C58470BD0028186811D00019408880067A
S3151C003EC08016FFF765FE116882268E57B042EEDA21
S3151C003ED018680019408880068016401C10E00019DE
S3151C003EE0408880068016FFF753FE116882268E577F
S3151C003EF0B042DCDD18680019408880068016401E1A
S3151C003F00FFF735F970BD0000FFFD0000840000209E
S3151C003F1080A2010090000020F7FF000080A0010095
S3151C003F200000003000010020F0B585B00020694675
S3151C003F30FE4F08723868818A09047DD403252D0733
S3151C003F40A98A2021C943A982F94C202122680D2661
S3151C003F507603921951845321095C002911D026211C
S3151C003F60415E10311F2902D9C07D80070DD42068FF
S3151C003F70F04942182820105E226880025118498D8B
S3151C003F800CE002A8FEF737FF0AE02068E949421850
S3151C003F902C20105E226880025118C98DC9B20843B4
S3151C003FA0009001A8FFF74CF90390E04807683846D3
S3151C003FB03A3001F016FF1021C8410099401888427A
S3151C003FC001D20020C04303990090012921D0F98C0D
S3151C003FD000291ED0D849897C090181427CD227221E
S3151C003FE001991202914205D8D44A914274D9F97D9D
S3151C003FF0490671D501A96846FFF7ECFECB4A116844
S3151C004000CB7DD807CE48085E20D000281CDA401C81
S3151C0040101FE001A96846FFF7DDFE6846007A002806
S3151C00402010D0002001218003C903411803984003C6
S3151C0040300143BE48006800E002E0027F1143818212
S3151C00404005B0F0BD0120EDE7002002E00028FBDDF5
S3151C004050401EC884980740D55320475C0120B94AA6
S3151C0040604002002F01D05F0705D5A98AAA822168C4
S3151C0040708919088166E0DB07FF27002B13D026234E
S3151C004080CB5E103312D13E20C043FEF7D3FC012079
S3151C004090FEF7D0FCA88AAF82012122688902A548B6
S3151C0040A0101881844EE0C98C0F2905D0A98AAA82D2
S3151C0040B0216889190881D8E73F20FEF7BBFC002040
S3151C0040C0C043FEF7B7FCA88AAF8201202268800293
S3151C0040D098495118888435E051E0944F58072DD5DE
S3151C0040E09806800F06D0012815D0022816D0032862
S3151C0040F028D117E02820085E042801DB012100E0F6
S3151C0041000021032802DB8007C00F01E0C007C00F97
S3151C004110FFF79AFE16E0D807C00F0DE0D807C00FB0
S3151C0041200121F5E7088D01218007C00FFFF78CFEE2
S3151C0041303868008DC007C00F0021E9E7C88C40B263
S3151C004140FEF70BFDFFF73DFE784800270068478702
S3151C0041508787FEF7DCFC02A8FEF74DFE0090A88AB6
S3151C0041602020C043A8822068801947846F480068B5
S3151C004170C18C027F4906490C0A43828260E7010C06
S3151C0041807987B887FEF7C3FCA88A2020C043A8827B
S3151C0041902168002089194884E8E7F0B50320000748
S3151C0041A0818AF021C9438182614AF02114680D235A
S3151C0041B05B03E418E180818A6349818214680021CB
S3151C0041C0E4182181848AE024E44384821468E41878
S3151C0041D02184848A3224E44384821468E41861842A
S3151C0041E0848A5A4D858216680D24F3185C85838A49
S3151C0041F0574B838214684F4BE4182180848A554E92
S3151C00420086821468E4186180848A86821468E4189D
S3151C004210A180848AB41C84821668F618F180868A6A
S3151C00422084821668F6183181868A84821468E4189A
S3151C0042306181848A484C84821468E418A181848A2A
S3151C004240AC11848221261768B602FF18FE81868A65
S3151C004250832686821668F6187182868A3F4E868267
S3151C0042601668F6183183868A7F2636028682166879
S3151C004270F6187183868A848231241668A402F6187D
S3151C004280B483848AFF24043484821468E418218449
S3151C004290848A81821468E4186184848A8182146801
S3151C0042A0E418A184848A81821468E318D984838AD9
S3151C0042B00823DB43838213681E4C40341B19198068
S3151C0042C0838A274B83821368264C1B195984838A3D
S3151C0042D0214BC13B83821468234BE4186180848A7A
S3151C0042E081821468E418E185848A81821468E41842
S3151C0042F02186848A81821468E4186186848A818274
S3151C0043001468E418A186848A81821468E418E186FC
S3151C004310848A81821468E4182187848A81821468BD
S3151C004320E3185987838A0A4E20361FE09000002026
S3151C0043308400002040A0010000040020CC070000DF
S3151C00434026000000FFFD000080810000E0FF000049
S3151C004350DF3F0000FD130000C0C00000FD0F000081
S3151C004360FFFB000080A1010080A401008682146866
S3151C004370F84BE418A181848A86821468E318998410
S3151C004380838A85821068F34A40328018C185F0BD45
S3151C004390032109078A8A00228A82EF4900020968DA
S3151C0043A00D22520389188030488370470322120756
S3151C0043B0938A3F23938209070001090F08430002D1
S3151C0043C0802140300843E44909680D2252038918AC
S3151C0043D04883704710B500221146E04C07E0C3071E
S3151C0043E002D04B00E35A5A40491C89B240080028A7
S3151C0043F0F5D1104610BDF0B5D748D94D00680D2132
S3151C00440049034018868B00273C4609E0385D290A7B
S3151C0044104840FFF7DFFF29024840641C85B2A4B25E
S3151C004420B442F3D32846F0BDFEB5CB4E31680D27FA
S3151C0044307F03C919498BCB4A090A146800252246F1
S3151C00444080320192C84A0300527DD2000092224655
S3151C004450A0320292603A01F0ADFD190E1918183FF0
S3151C00446067F8FAFFF4F3F2F1F018EFEEEDECEBEA75
S3151C00447018E918E8180003200007818AC021C943DF
S3151C004480818231688020C9194883FEBD002905D068
S3151C00449001290ED0022916D0012146E2907C002863
S3151C0044A0F3D00120607401980121807C01F0DDFAB3
S3151C0044B037E20198AB4C807C012101F0D6FA2168C9
S3151C0044C0012048742DE2507A01210843507265740C
S3151C0044D001980021807CE9E7002906D001290BD030
S3151C0044E0022913D00329E3D117E003200007818A90
S3151C0044F0858201F0ECF905E003200007818A85829C
S3151C00450001F0E1F93168C91988830AE20320000722
S3151C004510818A85820198807CF4E703200007818AC2
S3151C004520858201F00DFAEDE7891E0B0001F042FDB4
S3151C0045300524314B5D050400A7E7617C02295AD28C
S3151C004540D37C012B70D8937C002B01D100299CD0E5
S3151C00455011763068C019808BE084FEF702FD0100DD
S3151C00456001D006204FE07F480521006841740321D5
S3151C00457009078A8A8D822BE1907C002802D1607CF7
S3151C004580002882D0607C107601206074FFF70EFA3A
S3151C004590C7E1507A012108435072607C714E022893
S3151C0045A00AD37248704C0560714860812081411C99
S3151C0045B0704801F012FC6575FFF706FA3068582141
S3151C0045C0095C4174ADE1607C022811D2D17C0129C1
S3151C0045D02AD8917C002901D10028ADD0624901203E
S3151C0045E04875607C1076022018E0607C022803D394
S3151C0045F000990143C9B2ABE0D17C012914D8917C46
S3151C004600002905D102E0FFF7D1FEFEBD0028FCD033
S3151C004610554901204875607C107603206074FFF7AD
S3151C0046202FF9FEF774FA7CE1B1E045E111E109E1ED
S3151C004630D0E0E9E0D4E083E037E02DE021E018E0AB
S3151C00464012E00CE008E002E0FFE7605C1FE0306867
S3151C004650C019808B605464E14348405C17E03068A5
S3151C004660C019808B404A1EE0601840780202605CCC
S3151C0046700CE03068C019808B6054000A61184870C1
S3151C0046804FE1394842185278405C1202104303210C
S3151C00469009078A8A8D8235E73068C019808B324AB1
S3151C0046A0030A5418637050543BE1607C022844D2C0
S3151C0046B000290FD0012922D00229A6D12A482B492C
S3151C0046C045750D602A4941810181491C294801F023
S3151C0046D084FB30E0002300951A4611210220019527
S3151C0046E001F0B0FA2049012048754889204A088102
S3151C0046F0904201D1002000E0401C088111E11A4AB9
S3151C0047001C4811895389405C994203D1FF21013110
S3151C004710084306E0164B994201D1002100E0491CD2
S3151C0047201181032109078A8A8D823268C1B2D21986
S3151C0047309183000A67D0012081E00021052062E7F1
S3151C004740607C8446022817D3009861460843C1B290
S3151C0047500C2058E7C0A4010084000020AE3F0000D6
S3151C004760FFFF0000900000200004002088000020AD
S3151C004770FF02000000010020480705D53368F848F1
S3151C0047801B185B8EDB0705D0D07C012809D90221BA
S3151C0047900D2038E731680818408EC107C90F08205C
S3151C0047A031E7907C002803D16046002800D12CE715
S3151C0047B0EC4B01205875607C107604206074E17502
S3151C0047C0FFF752FA03200007818A8582E6480068B3
S3151C0047D0C08C97E6507A01210843E34E5072E0E6FE
S3151C0047E09088A17D4118E148405C032109078A8A0B
S3151C0047F08D823168C9198883A07DBF2801D300200A
S3151C00480000E0401CA0758CE09188A07DD74A0B184F
S3151C004810D35CBF2801D3002000E0401CC0B2A075A9
S3151C0048200918515CBF2801D3002000E0401CA0756C
S3151C00483003200007828A85821802084362E6FFF776
S3151C004840A7FDFEBD03200007818A8582FFF7D3FDE5
S3151C00485058E60298C44E41704806400F012817D0EE
S3151C004860022803D0052835D00628EAD1607C022808
S3151C00487000D3BDE6917C002901D10028E1D0B949BD
S3151C00488001204875617C11766074FEF765FD48E071
S3151C004890607C002847D006206074FEF7E7FD40E0E8
S3151C0048A0A582FEF787FF3068014640310A7E4274B6
S3151C0048B0A03045700D7634E03068C019408B0299E3
S3151C0048C0000A4870A84E4006400F12D0012821D07D
S3151C0048D00228B6D1607C0228E2D3A548A14F056008
S3151C0048E0A44878813881411CA04801F076FA7D7570
S3151C0048F0D6E7607C0228BCD2917C002901D1002815
S3151C0049009FD0984901204875617C11766074FEF72A
S3151C00491078FF06E0607C002805D007206074FEF74F
S3151C00492079FF00208BE70098C1B201206BE630B5F9
S3151C0049308D490020096808860C464886403420723A
S3151C004940627A0B46520852006272A072E0722073A1
S3151C0049508033D873834AA073927FE2730A4660320F
S3151C0049602074D075187158710887C8862075A07573
S3151C004970107150715872E07748859071D071107221
S3151C0049808885C88550721075D07450759075507690
S3151C0049909076D0761077987518760125DD7560802F
S3151C0049A058769876D876488248738873C873087484
S3151C0049B050779077D077187010769871888618740F
S3151C0049C088828875C8750883488330BD10B5FFF783
S3151C0049D0E4FBFFF7ACFF644800688079C0070BD185
S3151C0049E003200007818A0F21C94381826249002066
S3151C0049F00968624A8918488000F0F8FA10BD70B53B
S3151C004A0000F065FF574AD188002914D0CB08C01A7C
S3151C004A100818D080107B012114280ED2584B594DF2
S3151C004A2043435B199B12D4885B1C5B109C4204DCC1
S3151C004A30D174401C0FE0C000EBE700280DD0504B92
S3151C004A40514D43435B199B12D4885B1C5B109C42E3
S3151C004A5003DBD174401E107370BD0020D07470BD72
S3151C004A6070B526213F4801F0B8F93E4C262020801F
S3151C004A704648A0800B20A07300262073E67426757A
S3151C004A80667500F024FFC000E0800025FFF7B7FF25
S3151C004A906D1CEDB2082DF9D3374A1068304B403BDC
S3151C004AA0C018C08F28210007000FE0732674012050
S3151C004AB06073A1750421E175102121766676A076B6
S3151C004AC00221E17603212177242161772021A17718
S3151C004AD00521E677C90121840B2189016184032103
S3151C004AE009078D8A0F25ED438D8212680F21D21876
S3151C004AF051841C49203108715F21C9001B4801F0F3
S3151C004B006CF91B4806601B4860812081411C1748B4
S3151C004B1001F063F970BD1448002100680A2302469F
S3151C004B20018040329371D171C172817201734173DC
S3151C004B3081730174C17341824174917401718171D5
S3151C004B40C171017241724177022242710122827047
S3151C004B50024680321172D177A0300170E7E6000060
S3151C004B6080A101000004002090000020000100200C
S3151C004B7088000020FF0200008400002080A00100A5
S3151C004B809956FCFFE6F7D3005A60DA0002D1000002
S3151C004B9070B5694D2868694E8019C18E28688019C0
S3151C004BA0008F8A044B05520F5B0FD21889065208D8
S3151C004BB0890E51188204530FC206D20E9B18840903
S3151C004BC0E40700D05B424405640FA2184009C007E5
S3151C004BD000D052429818431028688019408F8006CE
S3151C004BE0841628688019408F4005C21628688519C6
S3151C004BF03A20285EC012002900DA4942002B00DA4E
S3151C004C005B42C918002C00DA64420919002A00DA32
S3151C004C1052428918002800DA4042081880B270BD3A
S3151C004C20F0B5454D2868454A8018C18E28688018FD
S3151C004C30008F2B689B185B8F5B05DB121C0C2B688B
S3151C004C409B183A229A5E8B044E055B0F760F9B19B6
S3151C004C5089065B08890E5E188104C3065201490F3A
S3151C004C60DB0E120CC9188709FF0700D049424705FD
S3151C004C707F0FFB184009C00700D05B42C818296883
S3151C004C8043102E480818408F8006811648005D1870
S3151C004C908446401965002A4C4019246880182488CB
S3151C004CA000B2A706BF0F022F09D1640707D558000B
S3151C004CB080194118604608184019801800B2F0BDCA
S3151C004CC000B5FFF765FF81004000081880B200BDE3
S3151C004CD000B50022FDF738FF002801DA4042012208
S3151C004CE015490968154B4033C9180988C908C907ED
S3151C004CF0C90F02D04000134902E012494000403956
S3151C004D00085E002A01D0404200B200BD10B5032146
S3151C004D1009078A8A8A138A82074A80061468C30D81
S3151C004D2006482418E3828B8A074B8B821268591C0F
S3151C004D301018C18210BD00008400002040A0010094
S3151C004D4090000020FE3F0000FF7F000030B50322CC
S3151C004D501207938AFE4B93824402FE480568FE4B5B
S3151C004D60ED18EC82948A7F24640294820468E41809
S3151C004D70E182918AF949918205684C1CED18EC82F6
S3151C004D80948A918200680021C018C18230BDF0B59A
S3151C004D9003200007818AF2498182EE4901230C68AF
S3151C004DA05B03F04AA418E381838AEF4B83820123B9
S3151C004DB00C689B03A418E381838AEB4B80338382A4
S3151C004DC009230C685B02A418E382838AE74D85825B
S3151C004DD00E681424E34B4033F6183484868A858285
S3151C004DE00E68F6187484848AE14C848201260F6846
S3151C004DF07602FF183E84878A84820F68FB185E84BD
S3151C004E00838A85820D680023AD186B82858A84820D
S3151C004E100D68AD186B82858A848208688018838227
S3151C004E201124E0B20021FFF791FF641C182CF8DB5B
S3151C004E30F0BD70B503242407A08AC848A082C54DBE
S3151C004E40401C2968C74E8919C881A08A3F20C043C7
S3151C004E50A08229681420C04A8918C8811F20FFF720
S3151C004E6055FFA08A0F20C043A08229680420BA4A95
S3151C004E70403289184880A08A7F20C043A0822968B6
S3151C004E80242089190883A08ABA48A08201222B688B
S3151C004E909203B44940315B181A84A38AA0822B68FA
S3151C004EA05B185A84A28AA0822B68002259188A840D
S3151C004EB0A18AA082296889194A82A18AA0822868A7
S3151C004EC08019828270BD10B503200007818AA6490D
S3151C004ED08182A04A00231468A24964186384838AC9
S3151C004EE09E4B83821268581C5118488410BD10B5FD
S3151C004EF0032109078A8A9F4A8A8282029548036887
S3151C004F00984C1B199A828A8A9B4A8A8205230468B2
S3151C004F105B02914AA41863828B8A984B8B82072367
S3151C004F2004685B03A41863828B8A2023DB438B8271
S3151C004F3004682023A41863828B8A1023DB438B828C
S3151C004F4004681023A41863828B8A4023DB438B825C
S3151C004F5004680023A41863828C8A0C24E4438C8284
S3151C004F6000688018438210BD70B5032109078A8A20
S3151C004F70804A8A828202774803687A4C40341B191D
S3151C004F809A848A8A754B8B8205685C1C724AAD189A
S3151C004F902C838C8A8B8204680023A41863838C8AD6
S3151C004FA0774C8C820468A41823838C8A754C8C825B
S3151C004FB00468A41823838B8A0223DB438B82046830
S3151C004FC00223A41823838C8A0F24E4438C8204684E
S3151C004FD0A41863838B8AF023DB438B820068202111
S3151C004FE0801841830020FEF725F870BDF0B503201C
S3151C004FF00007818A5C498182564901230C689B0300
S3151C005000584AA2189384828A544B83820C685D1C6E
S3151C005010544AA2189584828A7F22520282820E6882
S3151C00502000244D4AB618F482868A494E86820F6839
S3151C005030AE11BF18FE82868A83820E68B618F58268
S3151C005040868A83820E68B618F482868A404E8682C9
S3151C0050500F686E11BF18FE82868A83820E68B61888
S3151C005060F582868A83820E68B618F482868A384E42
S3151C00507086820F68C614BF18FE82868A83820E68D3
S3151C005080B618F582868A83820E68B618F482868ADA
S3151C0050902F4E86820F682E11BF18FE82868A838247
S3151C0050A00E68B618F582868A83820E68B618F48254
S3151C0050B0868A274E868205260F687602BF18FE82D0
S3151C0050C0868A83820E68B618F582868A83820E6863
S3151C0050D0B618F482868A1E4E86820F688614BF18FE
S3151C0050E0FE82868A83820E68B618F582868A838239
S3151C0050F00E68B618F482868A154E868207260F68B5
S3151C0051007602BF18FE82868A83820E68B618F582DE
S3151C005110868A83820E68B618F482868A0C4E86822C
S3151C0051200F68EE10BF18FE82868A83820E68B61838
S3151C005130F582868A83820E68B618F482868A044EA5
S3151C005140868209260F687602BF18FE82868A1BE0B5
S3151C005150FFC100008400002040A00100FF7F00006A
S3151C005160FFDF0000C0A40100FFBF0000E0FF00003D
S3151C0051701FFC0000FF830000FFF00000FF0F000073
S3151C005180FF9F0000FFEF000083820E68B618F582B1
S3151C005190858A83820D68AA18D482828AFE4A8282F4
S3151C0051A00D68FE4AAA189484828A83820968FB4881
S3151C0051B008188484F0BDF8B51F20FFF7A7FD03244B
S3151C0051C02407A08A0F20C043A082F54E0720316811
S3151C0051D0F44D49194880A08A7F20C043A0823268BA
S3151C0051E02221EE48101801830020FDF723FFA08A18
S3151C0051F00820C043A08231680820491908801E2057
S3151C005200FDF7ABFC1125E8B20021FFF79FFD6D1CD5
S3151C005210172DF8DBA08AF020C043A082E048C021ED
S3151C00522000680D277F03C019C180A08ADE48A082B2
S3151C005230DB4A012113688903D84A40329B1819841A
S3151C005240A38AA082D64B1B689A185184A18AA08275
S3151C005250D34800250168D148081845822846FFF71F
S3151C00526046FED2481921006860300170A08AD04ED3
S3151C005270A682CB48711C0268CA4840381218118392
S3151C005280A18AA682C649096809184D83A18AA682E5
S3151C005290C349096809184D80A18AA682C0490968B4
S3151C0052A009188D80A18AA682BD4909680918CD8076
S3151C0052B0A18AA682BA49096809180D81A18AA68203
S3151C0052C0B7490968081845811020FFF74DFEA08ACA
S3151C0052D02020C043A082B24920200968C91908842D
S3151C0052E0A08AE81EA082AE480068C0194584A08A20
S3151C0052F0A81EA082AA4801250068C0194584AD488D
S3151C00530000F0EBFAA6480068A44940394018808F83
S3151C005310C00703D000F005FB00F0F4FAA3480022F6
S3151C00532000689F210A54A0210D549D490B689D4D70
S3151C00533080355B19DB8A1B071B0F4030C374A08AA0
S3151C005340A6820B6895481B185A84A28A924AA28286
S3151C00535001220968920308184284F8BDF0B503209F
S3151C0053600007818A924C84828D4900230D688D4AE0
S3151C005370403AAD182B83858A84820D68AD186B83E1
S3151C005380858A84820E68651CB6187580868A848216
S3151C0053900E68B618B580868A84820E68B618F580A3
S3151C0053A0868A84820E68B6183581868A84820E683F
S3151C0053B0B6187581868A84820C68A4182580848A0E
S3151C0053C0754C84826C100D68AD182C80848A7A4EBC
S3151C0053D086820D680224AD186C80858A86820D68CB
S3151C0053E0AD18AC80848A3F24E44384820C68202751
S3151C0053F0A418A781848A714C84820D683C02AD185E
S3151C005400AC81848A6E4C84820D68AD186B80858A4B
S3151C0054106C4D85820E68B6187380868A84820E68E7
S3151C005420B618B380868A85820E68B618B380868ABB
S3151C00543084820E68B618F380868A85820E68B61832
S3151C005440F380868A84820E68B6183381868A8582A2
S3151C0054500E68B6183381868A84820C68A418638108
S3151C005460848A85820C68A4186381838AFB438382A1
S3151C005470086880180780F0BDF0B503242407A08AAD
S3151C0054804B4EA682464D00202968464F403FC919FF
S3151C0054900883A08AA68229680020C9194883FFF7B9
S3151C0054A05DFFA08A4048A0820120296880033B4AF0
S3151C0054B0403289188884A08AA6822968701CC9195A
S3151C0054C04880A08A4020C043A0822A6840210D2023
S3151C0054D0400312181184A18A2021C943A1822A687B
S3151C0054E0002110180184F0BD70B503242407A18A7D
S3151C0054F02D49A1822A4D80022968284A40328918E2
S3151C0055008884A08A2A4AA2822B6800212548403812
S3151C0055101B181983A38AA2822B68521C1B185A8338
S3151C005520A28A274AA2822A6812181183A28A264AAC
S3151C005530A2822A6812181183A18A0221C943A18258
S3151C0055402A68022112181183A28A0F22D243A28230
S3151C0055502A6812185183A18AF021C943A1822A689C
S3151C005560202112185183A18A1849A1821F222B6857
S3151C00557092021B189A83A28AA18219212A6889027F
S3151C0055801018C1810020FDF755FDA08A0820C043D4
S3151C005590A082082029681BE0FFBF0000C0A40100F0
S3151C0055A08400002080A00100FF83000090000020E2
S3151C0055B0FF7F0000A0860100FDFF0000FFC0000069
S3151C0055C0FF9F0000FFF30000FFEF0000FF03000039
S3151C0055D0AB4A8918088070BDF8B5FFF779FBA94C52
S3151C0055E02168C884FFF76CFB2168A74C4884226895
S3151C0055F0A34840381018808E03258006800E02466C
S3151C005600143A00272D070C2AA04EAA8AAF822268BC
S3151C00561014D3921950861428A88AAF82206806D201
S3151C0056208019808E22689219401C908613E080197E
S3151C005630C08E22689219401CD0860CE092191086E6
S3151C005640AA8AAF8222689219D28D23689B19521C92
S3151C005650DA85602250542620085E4A8C82188C48B3
S3151C005660008C82420EDA2368854840381818808ED2
S3151C005670C00B07D10B46603318781F2802D2401C7A
S3151C005680187013E08248408C82420FDD22687C48E9
S3151C00569040381018808E800BC007C00F06D10A46F2
S3151C0056A060321078142801D9401E107060310878B9
S3151C0056B0FFF72CFBA88AAF8272482168006860300D
S3151C0056C0007889190887A88AAF8220688019408FBC
S3151C0056D021688919401C4887F8BD70B56A4D286831
S3151C0056E0674E80194088674C01072068090F603097
S3151C0056F08170FFF795FA082807DD216860318A78E2
S3151C0057000F2A02D2521C8A7009E00821C84206DA06
S3151C005710216860318878002801D0401E88700320DB
S3151C0057200007818A0F21C94381822068296860305D
S3151C00573080788919488070BDFEB5524F02263A689A
S3151C0057404032907A01280CD0002502280BD039460D
S3151C00575009688031032803D0042800D08D774D7743
S3151C0057600D779672FEBD03242407A08A494BA3829B
S3151C005770454D00202A684249403952181083A28A96
S3151C005780A3822A6851184883FFF7E8FDA08A42487D
S3151C005790A0820120296800033C4A8032891888842B
S3151C0057A0A08A4020C043A0822A6840210D204003C5
S3151C0057B0101801843868012402468030017F491C78
S3151C0057C0C9B2017700290ED0FFF706FF38680325FA
S3151C0057D002468030417F491CC9B24177022905D255
S3151C0057E040329572FEBD40329472FEBDFFF775FFC6
S3151C0057F0386802468030817F491CC9B281770229EC
S3151C00580003D2042040329072FEBD00F0A5F8002899
S3151C00581013D000F086F8214800F05FF800F072F80B
S3151C005820386801468030C477807C4031897A000113
S3151C00583040180006000CF1210BE038680146803048
S3151C005840C577807C4031897A000140180006000C1F
S3151C005850E3210843019000230222322100960120F5
S3151C00586000F0F0F903200007818A2021C9438182B8
S3151C0058700548002102680D20400310180184FEBD56
S3151C00588080A00100900000208400002080A401005C
S3151C00589000040020FF7F0000FF830000A08601009B
S3151C0058A034480079C007C00F7047324801788F22F0
S3151C0058B01140017001790178012211430170704772
S3151C0058C02C48806870472B48008980B2704703209B
S3151C0058D00007008A8005800D7047274909688031BA
S3151C0058E0897C0907090E8A002249403151188860B3
S3151C0058F008788F2210401030087008780122104357
S3151C005900087070471C4800688030807C0007000EB9
S3151C0059108100184840300818017802221143017092
S3151C0059207047154800688030807C0007000E810097
S3151C0059301048403008180178FD221140017070474C
S3151C0059400D480C49006840318030807C0007000EF1
S3151C00595080004018C06870470748064900684031F7
S3151C0059608030807C0007000E800040180079C0073C
S3151C005970C00F7047C00000309000002010B572B6F2
S3151C0059805849C869FF22120490430122920510430C
S3151C005990C86156495448486088600020544A012111
S3151C0059A0C406E40E0B46A3404409A400A4182360B5
S3151C0059B0401C40B20C28F3DB62B610BD10B50022A9
S3151C0059C01146019800F0A4F810BD10B5002211462E
S3151C0059D0019800F09DF810BD10B5002211460198E3
S3151C0059E000F096F810BD10B500221146019800F083
S3151C0059F08FF810BD10B500221146019800F088F8EA
S3151C005A0010BD10B500221146019800F081F810BD9A
S3151C005A1010B500221146019800F07AF810BD10B599
S3151C005A2000221146019800F073F810BD3148407EE3
S3151C005A30C4E73048807EC1E72E48C07EBEE72D48AD
S3151C005A40007FBBE72B48407EBFE72A48807EBCE729
S3151C005A502848C07EB9E72748007FB6E710B5002264
S3151C005A601146019800F054F810BD70B5214B024642
S3151C005A705D7E04200824954210D09D7E954202D15D
S3151C005A80052009240AE0DD7E954202D106200A245F
S3151C005A9004E01B7F934201D107200B24002905D06B
S3151C005AA000F014F8204600F011F870BD00F004F860
S3151C005AB0204600F001F870BDC206D20E01219140AD
S3151C005AC040090D4A8000801801607047C206D20E3C
S3151C005AD001219140084A40098000803280180160EB
S3151C005AE07047000004ED00E08080808000E400E048
S3151C005AF080E200E00004002000E100E010B5202157
S3151C005B003E4800F06CF920213D4800F068F910BDB4
S3151C005B1072B6BFF3408F032109078A8A00238B8242
S3151C005B20394A38491268394C1219D1863849202409
S3151C005B300A7C22430A74EFF30581304A8906890ED2
S3151C005B4014781170002C0DD191709060EFF30880C1
S3151C005B50D060EFF309801061EFF306809061EFF3DC
S3151C005B600380D0610120102906D3054610395469DB
S3151C005B708D402C43546104E0054654688D402C43EB
S3151C005B8054605370BFF3408F62B6D1780143D17015
S3151C005B90FEE7F0B5059D72B6BFF3408F1C4C40273F
S3151C005BA0267C3E432674164C26782070002E09D17E
S3151C005BB0A070A160EFF30881E160EFF30981E56154
S3151C005BC0A36121610121202806D30D462038636973
S3151C005BD085402B43636104E00B46656883401D4387
S3151C005BE0656000206070BFF3408F62B6002A03D048
S3151C005BF0E0780843E070FEE7F0BD000028040020B2
S3151C005C0048040020ADDE00008400002080A40100B2
S3151C005C1000040020F0B54C4D0A21695E00224B4E53
S3151C005C204B4B4C4F0AE0B45C5C54401E521C491E44
S3151C005C3009B2C0B2D2B2002900DA39460028F2D124
S3151C005C406981F0BDFFB581B0054604980B9E0028FE
S3151C005C5000D172B63C49487BFF2802D14B89082BE0
S3151C005C6001D3012400E00024029B5B1EFD2B52D2B3
S3151C005C70002C50D03449497D00294CD1012D02D02D
S3151C005C80002D03D004E0344800684079904242D38A
S3151C005C90FFF716FE0746010C30480068000C081A70
S3151C005CA00004000C12D02949FF228A70020A4A708D
S3151C005CB008700320FFF7AEFF2348417BFF2904D160
S3151C005CC04089082801D2002400E001242348002C26
S3151C005CD0076020D0012D24D0002D27D008240A9837
S3151C005CE0002808D01948310A06704170310C8170A1
S3151C005CF00A98FFF78FFF0A981449001D400120439C
S3151C005D00C87016480088020A8A7048700298087083
S3151C005D100420FFF77FFF0498002800D162B605B067
S3151C005D20F0BD0D4800688030847CD8E70F24D6E788
S3151C005D301CB50A46002100910B4601910146012023
S3151C005D40FFF780FF1CBD0000000400208C00002013
S3151C005D5000010020FF0200009000002088000020A7
S3151C005D6030B50E49002009780B4D4C1E11E002027D
S3151C005D70521980329074002805D0431E1375A04218
S3151C005D8003D1002302E02346F8E7431C401CD374CE
S3151C005D90C0B28842EBD330BD000500208000002035
S3151C005DA0704701E004C0091F0429FBD28B0701D5EB
S3151C005DB00280801CC90700D00270704700290BD0D6
S3151C005DC0C30702D00270401C491E022904D3830754
S3151C005DD002D50280801C891EE3E70022EEE7002222
S3151C005DE0DFE70378C2781946437812061B0219436B
S3151C005DF08378C0781B04194311430902090A00065B
S3151C005E0008437047002203098B422CD3030A8B429A
S3151C005E1011D300239C464EE003460B433CD4002280
S3151C005E2043088B4231D303098B421CD3030A8B4292
S3151C005E3001D394463FE0C3098B4201D3CB01C01A60
S3151C005E40524183098B4201D38B01C01A524143092B
S3151C005E508B4201D34B01C01A524103098B4201D319
S3151C005E600B01C01A5241C3088B4201D3CB00C01A86
S3151C005E70524183088B4201D38B00C01A52414308FE
S3151C005E808B4201D34B00C01A5241411A00D2014623
S3151C005E905241104670475DE0CA0F00D049420310BC
S3151C005EA000D34042534000229C4603098B422DD30B
S3151C005EB0030A8B4212D3FC22890112BA030A8B42B3
S3151C005EC00CD3890192118B4208D3890192118B4202
S3151C005ED004D389013AD0921100E08909C3098B4287
S3151C005EE001D3CB01C01A524183098B4201D38B01CA
S3151C005EF0C01A524143098B4201D34B01C01A52416D
S3151C005F0003098B4201D30B01C01A5241C3088B42B1
S3151C005F1001D3CB00C01A524183088B4201D38B009C
S3151C005F20C01A5241D9D243088B4201D34B00C01A26
S3151C005F305241411A00D20146634652415B1010463B
S3151C005F4001D34042002B00D54942704763465B1083
S3151C005F5000D3404201B50020C046C04602BD704772
S3151C005F60754600F023F8AE46050069465346C00840
S3151C005F70C000854618B020B5FCF777F960BC002731
S3151C005F804908B6460026C0C5C0C5C0C5C0C5C0C5E3
S3151C005F90C0C5C0C5C0C5403D49008D4670470446B6
S3151C005FA0C046C0462046FCF746F90000004870472C
S3151C005FB09400002030B47446641E2578641CAB42E1
S3151C005FC000D21D46635D5B00E31830BC18472110E8
S3151C005FD042208440088131126224C4488891000002
S3151C005FE00A0015001F00290034003E00490053001A
S3151C005FF05D00680072007C00870091009B00A60073
S3151C006000B000BA00C500CF00DA00E400EE00F900CB
S3151C00601003010D01180122012C0137014101000069
S3151C0060201100230034004600570069007A008C00DA
S3151C0060309D00AF00C000D200E300F5000601180168
S3151C00604029013B014C015D016F0180019201A301F5
S3151C006050B501C601D801E901FB010C021E020000B4
S3151C006060604000008000002014000000C4010000F5
S3151C00607074400000940000206C080000E001000041
S3151C00608000000000000000000000000000000000EE
S3151C006090000000000018000010402DE90040A0E19F
S3151C0060A0B8039FE5004080E5000090E5500080E2C3
S3151C0060B0AC139FE5000081E5A0039FE5000090E579
S3151C0060C0650F80E29C139FE5000081E50800A0E3B4
S3151C0060D094139FE5000081E50000A0E37C139FE577
S3151C0060E0001091E5900181E570139FE5001091E584
S3151C0060F0940181E564139FE5001091E5980181E503
S3151C00610058139FE5001091E5200081E54C039FE59F
S3151C006110000090E5000090E550139FE5010050E15A
S3151C0061200500001A34039FE5000090E5040090E585
S3151C0061303C139FE5010050E10B00000A001200E32E
S3151C00614018039FE5000090E5C0E8FFFA1C039FE5D5
S3151C00615008139FE5001091E5000081E510039FE5FB
S3151C006160F8129FE5001091E5040081E51080BDE85A
S3151C006170E8129FE5000081E5001091E5901081E290
S3151C006180DC229FE5001082E5D0129FE5001091E508
S3151C006190661F81E2CC229FE5001082E51010A0E369
S3151C0061A0C4229FE5001082E51EFF2FE1AC029FE58D
S3151C0061B0000090E50C0090E5010080E29C129FE532
S3151C0061C0001091E50C0081E51EFF2FE18C029FE576
S3151C0061D0000090E5100090E5010080E27C129FE52E
S3151C0061E0001091E5100081E51EFF2FE16C029FE572
S3151C0061F0000090E5140090E5010080E25C129FE52A
S3151C006200001091E5140081E51EFF2FE14C029FE56D
S3151C006210000090E5180090E5010080E23C129FE525
S3151C006220001091E5180081E51EFF2FE12C029FE569
S3151C006230000090E5980190E520129FE5001091E57D
S3151C006240A00181E51EFF2FE110129FE5001091E5CC
S3151C006250A00181E51EFF2FE100029FE5000090E5ED
S3151C006260A00190E5F4119FE5001091E5980181E5E8
S3151C0062701EFF2FE110402DE9E0019FE5000090E58F
S3151C006280081080E20100A0E3E7E7FFEB1080BDE801
S3151C00629070402DE90040A0E1C0119FE5001091E57A
S3151C0062A09C0191E50510A0E3EDE8FFFA0150A0E181
S3151C0062B0A8019FE5000090E5240080E2054180E7E7
S3151C0062C098019FE5000090E59C0190E5010080E2A5
S3151C0062D088119FE5001091E59C0181E57080BDE861
S3151C0062E010402DE90040A0E178019FE5000090E5F3
S3151C0062F0000090E570119FE5001091E5011041E248
S3151C006300010050E10700009A58019FE5000090E546
S3151C006310000090E5000884E140119FE5001091E51E
S3151C006320200081E5150000EA38019FE5000090E594
S3151C006330000090E528119FE5001091E5804181E75A
S3151C00634020019FE5000090E5000090E510219FE5E7
S3151C006350002092E5800182E0041080E20100A0E3A7
S3151C006360B1E7FFEBFC009FE5000090E5000090E51F
S3151C006370010080E2EC109FE5001091E5000081E52C
S3151C0063801080BDE8D4209FE5002092E5902192E57F
S3151C006390080052E30700003AC0209FE5002092E562
S3151C0063A0902192E5022880E1B0309FE5003093E50C
S3151C0063B0202083E5150000EAA0209FE5002092E539
S3151C0063C0902192E594309FE5003093E5153E83E2DB
S3151C0063D0820183E784209FE5002092E5902192E5C7
S3151C0063E078309FE5003093E5153E83E2822183E0F9
S3151C0063F0041082E564209FE5002092E5902192E539
S3151C006400012082E254309FE5003093E5902183E51C
S3151C0064101EFF2FE110402DE940309FE5003093E52B
S3151C0064201C3093E50F2003E20030A0E11138DFE7B2
S3151C00643028409FE5004094E5114E84E2023184E732
S3151C00644018309FE5003093E51C3093E5013083E25C
S3151C00645008409FE5004094E51C3084E51080BDE8AB
S3151C0064600000040004000400080004000C000400E2
S3151C00647043415254474F4C450000000000000000A9
S3151C00648000000000000000000000000000000000EA
S3151C00649000000000000000000000000000000000DA
S3151C0064A000000000000000000000000000000000CA
S3151C0064B000000000000000000000000000000000BA
S7051C000000DE
